:1000000088C0B2C068C3B0C0AFC0B3C0ADC0ACC0E0
:10001000ABC0AAC0A9C0A8C068C1A6C0A5C0814580
:1000200086468B479048944997609B619E62A16386
:10003000A464A765AA66AC67AE68B069B280B481F3
:10004000B682B883BA84BB84BD84FF21000000005F
:100050000000000000000000000023456C98C9FF6C
:10006000040714233764A0FFFFFFFFFFFFFFFFFF1C
:10007000FFFFFF00000000000000000023405F7A47
:10008000B4FFFFFFFFFFFF001400081400080E1468
:100090000004080E14000305080E14000305080AE6
:1000A0000E14000305080A0E1014000305080A0EBA
:1000B0001012140008000E00080E0004080E0003C1
:1000C00005080E000305080A0E0004080E101400AF
:1000D000F3F404080E10121400080A0C0E0F10128C
:1000E0001400080EEE1400020304050004140004BA
:1000F0000E1400040810140004080F111400EEED93
:10010000ECEB140E08040004080E00EBECEDEEF32B
:10011000F41411241FBECFE5D2E0DEBFCDBF20E036
:10012000A0E6B0E001C01D92A938B207E1F7E2E60F
:10013000F0E085E5808781E08383148212828683E4
:100140001182AEE6B0E08EEF15968C9315978DEF89
:1001500017968C938BE0828788E58387612C712CBE
:1001600088248A94C3D00DC34BCF1BBC19BC18BCC8
:100170000895189525B7277E25BF29B7226029BF86
:1001800021E022BF019728F020E188952150E9F76E
:10019000F9CF089588EE93E0EDCF8CE287B986EC35
:1001A00086B9369A3699FECF8FEF80936000089516
:1001B000369A3699FECF95B18091600089270895CF
:1001C000CF93C72D81E0870D8F73782E662D90E039
:1001D000CAD26FEF8C2F90E0CF91C5C2FF920F93E0
:1001E0001F93CF93DF93F82E0DE610E0C4E7D0E025
:1001F00081E0F81205C0F8016081CE01B4D204C0DC
:10020000CE01A9D2F8018083015011092196CF3780
:10021000D10571F7DF91CF911F910F91FF90089554
:10022000CFDF81E0DBCF811101C09FCF815090E013
:10023000FC01E45BFF4FE491EBBDFC01E05AFF4F92
:10024000E491E9BDFC01EC58FF4F849188BD08950D
:100250000F931F93CF93C82F8B01CC2359F085E0C8
:10026000E2DFC80187DF81DFC80184DFC80182DFE8
:10027000C150F3CFCF911F910F910895EF92FF924C
:100280000F931F93CF93C8E0E82EF12C062F10E0B8
:1002900084E1C9DFC7016EDF68DFC8016BDFC150D1
:1002A000B9F7CF911F910F91FF90EF9008951F9391
:1002B000CF93DF938FEA87B986EC86B910926000FE
:1002C00010E1C0E0D0E085E090E054DF71DFC80FBE
:1002D000D11D1150C1F7CE0124E0969587952A953E
:1002E000E1F7DF91CF911F91089518958FEF881254
:1002F00010C083EA87B986EC86B93699FECF369A64
:100300003699FECF85B1833D18F086E0882E01C076
:10031000812C8FE384BBB99AB89ABC9A81E08ABDDC
:1003200083BF9AB590629ABD9AB590689ABD9FEFC7
:100330009DBD80BF80E68CBD97B328B3892F90E028
:10034000809590958B7F822B88BBAB9A8BB7806210
:100350008BBF8AB785608ABF85B7806285BF789476
:1003600087E790E0F8D1853511F05ADF11C0712C84
:10037000872D90E0F0D1682E8F3F19F080E02EDFBE
:1003800007C0872D91E0970D792E803488F3F6CF42
:1003900080916C001091650000916600C09163002F
:1003A000CC2319F000E010E088E18F5F90E040E09E
:1003B00050E068E870E0882379F09B012F5F3F4FA1
:1003C000F9013197E491EE2319F0922F961BF6CFA5
:1003D0008150AB01B901EFCF892F612F70E0A92FB8
:1003E000B0E0E82FF0E0002321F09D012E1B3F0B31
:1003F00005C09F0121503109260F371F3197E40FA7
:10040000F51FF49028583F4FF901F082815049F7C9
:10041000910F90936100112371F0002329F0292F8F
:1004200030E02150310902C020E030E0F901E85805
:10043000FF4F81E0808387E0890F282F2150E22F32
:10044000E91BF0E0E55FFE4FE491A22FB0E0A85871
:10045000BF4FEC932913F2CFE82FF0E0E958FF4F9C
:1004600021E0409178003081431320E0821B282F47
:1004700080938800862D853F78F5382D333060F4E1
:100480008F5F682E891708F0612C809189008F5F3B
:100490008F718093890020C0109289003630B0F4AB
:1004A00030916800332311F0CC2331F08F5F682E38
:1004B000891790F0612C10C06916E1F3662019F0DD
:1004C0008150682E09C02150622E06C0C111F2CFA2
:1004D00080916400882371F3812C72DE5EDEC62D6C
:1004E000C53F28F4D0E0C858DF4FC881DC2F10E0AA
:1004F00000E0EE24E39480918900803190F14ADE9F
:1005000010928900C3E6D0E0C12CD12C81E08C0D83
:10051000FFEFCF1ADF0A98819F3F31F4219689E0DF
:10052000C816D10499F718C06DE570E091DEF601A8
:10053000E259FF4F608088818E25888371DE6FE0ED
:1005400070E080E285DE88818E25888369DE22DE88
:1005500080916300882311F3612CC0917800DC2F17
:100560008EC0CE3E19F463E481E204C0CD3E21F496
:1005700068E284E183DE83C0CC3E11F469E203C00B
:10058000CB3E19F462E581E0F5CFC33F41F484E14D
:100590004ADE8AE090E0EEDD88E045DE3DC0C43F03
:1005A00059F584E690E0E6DDF8DD02DE90E0292FE3
:1005B00030E0F901E25EFF4FE491E81710F49E5F2E
:1005C000F6CFF901E15EFF4FF4906DE770E08F2DFB
:1005D0008295869587703CDE8EEE92E0CBDD65E0FD
:1005E00070E081E035DE85E694E0C4DD6DE770E023
:1005F0008F2D8F712DDE0FC0CE3F81F4612CF12C39
:10060000F0926C000DDE6AEF70E081E021DEF39481
:1006100098E1F912F5CFBEDDBDDD31C0CD3F91F4DB
:10062000612C8FEF80936D00FBDD85E0FCDDB2DD9A
:10063000B1DD84E1F8DD3BDE80936D00F1DDAADD04
:10064000A9DDF9CF8D2FEFDD32DE20916D0082170D
:1006500038F00F5F093078F0D33068F0D1500AC01D
:1006600090E030E022503109821793071CF4DC1728
:1006700008F4DF5F00E091DD84EF91E07BDD109214
:10068000890096DD803990F41F5F183008F433CF6D
:10069000D53120F010E0DAE0CAE02DCFD23040F0C2
:1006A0008D2F86958695D695D80FCD2F10E023CF28
:1006B0005CDD85B7877E806185BFF89485B78468E7
:1006C00085BF8B7F85BF85B7806285BF889585B7DD
:1006D0008F7D85BFEACF1124882009F01895F89402
:1006E00016B843DDB998B898BC9830E021E094E0A2
:1006F00086B38870222351F0811127C086E08815C7
:1007000010F021E0F5CF20E099E0F2CF332319F08B
:10071000882321F01AC031E0811130E085B7877E4F
:10072000806185BF892F887011F440E401C040E6E4
:10073000892F8770842B81BD85B7846885BF8B7FA7
:1007400085BF78948895F894D3CF8FE58DBF82E0EC
:100750008EBF1FBECBDDE199FECF9FBB8EBBE09A63
:1007600099278DB30895262FE199FECF1CBA9FBB20
:100770008EBB2DBB0FB6F894E29AE19A0FBE01969C
:060780000895F894FFCF7C
:00000001FF
